:020000040000FA
:0408000063EF09F0A9
:1008100003B283EF05F0F2B4A1EF05F09EB0A9EFAB
:1008200005F09EB2B1EF05F0F2A81AEF04F0F2B2B3
:1008300032EF04F09EB61FEF04F012EF09F09E961F
:1008400000011450000A06E000011450010A06E0FD
:1008500012EF09F057EC20F012EF09F04BEC22F008
:1008600012EF09F0CD90F2929EA03CEF04F001014E
:10087000533F3CEF04F0542BAEC1B2F1AFC1B3F122
:10088000B0C1B4F1B1C1B5F1AAC1AEF1ABC1AFF124
:10089000ACC1B0F1ADC1B1F1A6C1AAF1A7C1ABF134
:1008A000A8C1ACF1A9C1ADF1A2C1A6F1A3C1A7F144
:1008B000A4C1A8F1A5C1A9F19EC1A2F19FC1A3F154
:1008C000A0C1A4F1A1C1A5F19AC19EF19BC19FF164
:1008D0009CC1A0F19DC1A1F196C19AF197C19BF174
:1008E00098C19CF199C19DF1CECF96F1CFCF97F1F0
:1008F00053C198F154C199F1CF6ACE6A0101536B8B
:10090000546B9E90CD800FBC0F8E0FBA8BEF04F00E
:100910000F8A12EF09F00F8C0FBEC7EF04F096C1DB
:100920009AF197C19BF198C19CF199C19DF19AC12F
:100930009EF19BC19FF19CC1A0F19DC1A1F19EC1FF
:10094000A2F19FC1A3F1A0C1A4F1A1C1A5F1A2C1CF
:10095000A6F1A3C1A7F1A4C1A8F1A5C1A9F1A6C19F
:10096000AAF1A7C1ABF1A8C1ACF1A9C1ADF1AAC16F
:10097000AEF1ABC1AFF1ACC1B0F1ADC1B1F1AEC13F
:10098000B2F1AFC1B3F1B0C1B4F1B1C1B5F1010180
:100990005E6B5F6B606B616B96515E2797515F2357
:1009A00098516023995161239A515E279B515F238F
:1009B0009C5160239D5161239E515E279F515F236F
:1009C000A0516023A1516123A2515E27A3515F234F
:1009D000A4516023A5516123A6515E27A7515F232F
:1009E000A8516023A9516123AA515E27AB515F230F
:1009F000AC516023AD516123AE515E27AF515F23EF
:100A0000B0516023B1516123B2515E27B3515F23CE
:100A1000B4516023B5516123D89001016133603333
:100A20005F335E33D8900101613360335F335E33EF
:100A3000D8900101613360335F335E3300C10CF144
:100A400001C10DF102C10EF103C10FF104C110F19A
:100A500005C111F106C112F107C113F108C114F16A
:100A600009C115F10AC116F10BC117F134C135F1F5
:100A700011B846EF05F00101620E046F010E056F1B
:100A8000000E066F000E076F4FEF05F00101A70E75
:100A9000046F020E056F000E066F000E076F5EC139
:100AA00000F15FC101F160C102F161C103F1EEEC3F
:100AB0001EF003BF04D019BE02D019A0108C11A0E3
:100AC00067EF05F010BA67EF05F00F80108A0CC1D0
:100AD00000F10DC101F10EC102F10FC103F110C10E
:100AE00004F111C105F112C106F113C107F114C1DE
:100AF00008F115C109F116C10AF117C10BF135C191
:100B000034F112EF09F00392ABB2AB98AB8803015A
:100B100003EE00F080517F0BE92604C0EFFF802B2D
:100B20008151805D700BD8A48B8200008051815D63
:100B3000700BD8A48B9281518019D8B4079012EF12
:100B400009F0F2940101453F12EF09F0462B12EF34
:100B500009F09E900101533F12EF09F0542B12EF60
:100B600009F09E9211B820EF07F08BB4BFEF05F0AB
:100B700010ACBFEF05F08B84109CC0EF05F08B9498
:100B8000C3CF55F1C4CF56F1C28207B42AEF06F0A5
:100B900047C14BF148C14CF149C14DF14AC14EF139
:100BA0005EC162F15FC163F160C164F161C165F171
:100BB00096C1B6F197C1B7F198C1B8F199C1B9F131
:100BC0009AC1BAF19BC1BBF19CC1BCF19DC1BDF101
:100BD0009EC1BEF19FC1BFF1A0C1C0F1A1C1C1F1D1
:100BE000A2C1C2F1A3C1C3F1A4C1C4F1A5C1C5F1A1
:100BF000A6C1C6F1A7C1C7F1A8C1C8F1A9C1C9F171
:100C0000AAC1CAF1ABC1CBF1ACC1CCF1ADC1CDF140
:100C1000AEC1CEF1AFC1CFF1B0C1D0F1B1C1D1F110
:100C2000B2C1D2F1B3C1D3F1B4C1D4F1B5C1D5F1E0
:100C3000010155515B2756515C23E86A5D230E2E56
:100C40002AEF06F05CC157F15DC158F15B6B5C6B3C
:100C50005D6B078E0201002F12EF09F03C0E006F52
:100C60001A50E00BE00AE866128818BE02D018B4E9
:100C7000108E00C10CF101C10DF102C10EF103C1D2
:100C80000FF104C110F105C111F106C112F107C144
:100C900013F108C114F109C115F10AC116F10BC114
:100CA00017F134C135F101018A675EEF06F08B67F9
:100CB0005EEF06F08C675EEF06F08D6762EF06F080
:100CC00092EF06F08EC100F18FC101F190C102F1E7
:100CD00091C103F10101010E046F000E056F000EBA
:100CE000066F000E076FEEEC1EF000C18EF101C121
:100CF0008FF102C190F103C191F1006787EF06F017
:100D0000016787EF06F0026787EF06F0036792EF4F
:100D100006F08AC18EF18BC18FF18CC190F18DC12B
:100D200091F10F80D57ED5BE6DD0D6CF47F1D7CF0C
:100D300048F145C149F1E86AE8CF4AF119BE02D04D
:100D400019A0108C109047C100F148C101F149C1B0
:100D500002F14AC103F101010A0E046F000E056F92
:100D6000000E066F000E076FEEEC1EF003AF108052
:100D7000010154A7C8EF06F00F9A0F9C0F9E0101C6
:100D8000000E5E6F600E5F6F3D0E606F080E616F4C
:100D9000010147BFD8EF06F04867D8EF06F0496772
:100DA000D8EF06F04A67D8EF06F0F288FDEF06F0BC
:100DB000F2985E6B5F6B606B616B966B976B986B79
:100DC000996B9A6B9B6B9C6B9D6B9E6B9F6BA06BE7
:100DD000A16BA26BA36BA46BA56BA66BA76BA86B97
:100DE000A96BAA6BAB6BAC6BAD6BAE6BAF6BB06B47
:100DF000B16BB26BB36BB46BB56BD76AD66A0101DA
:100E0000456B466B0CC100F10DC101F10EC102F141
:100E10000FC103F110C104F111C105F112C106F1B6
:100E200013C107F114C108F115C109F116C10AF186
:100E300017C10BF135C134F112EF09F012EF09F0CF
:100E40000201002F79EF08F0D59ED6CF47F1D7CF1A
:100E500048F145C149F1E86AE8CF4AF1D76AD66A54
:100E60000101456B466BD58E1A50E00BE00AE8662F
:100E7000128818BE02D018B4108E17AE1C8C00C198
:100E80000CF101C10DF102C10EF103C10FF104C15A
:100E900010F105C111F106C112F107C113F108C12A
:100EA00014F109C115F10AC116F10BC117F134C1D2
:100EB00035F10FA0109A11B869EF07F00101620E29
:100EC000046F010E056F000E066F000E076F72EFC4
:100ED00007F00101A70E046F020E056F000E066FEA
:100EE000000E076F47C100F148C101F149C102F18D
:100EF0004AC103F1EEEC1EF003BF85EF07F019BE07
:100F000002D019A0108C11B00F800CC100F10DC1DE
:100F100001F10EC102F10FC103F110C104F111C1C1
:100F200005F112C106F113C107F114C108F115C191
:100F300009F116C10AF117C10BF135C134F10201F3
:100F40003C0E006F00C10CF101C10DF102C10EF1A8
:100F500003C10FF104C110F105C111F106C112F175
:100F600007C113F108C114F109C115F10AC116F145
:100F70000BC117F134C135F101018A67C7EF07F0E2
:100F80008B67C7EF07F08C67C7EF07F08D67CBEF74
:100F900007F0FBEF07F08EC100F18FC101F190C1A6
:100FA00002F191C103F10101010E046F000E056F02
:100FB000000E066F000E076FEEEC1EF000C18EF102
:100FC00001C18FF102C190F103C191F10067F0EF0F
:100FD00007F00167F0EF07F00267F0EF07F0036733
:100FE000FBEF07F08AC18EF18BC18FF18CC190F1BC
:100FF0008DC191F10F80109047C100F148C101F1FE
:1010000049C102F14AC103F101010A0E046F000E49
:10101000056F000E066F000E076FEEEC1EF003AFBB
:101020001080010154A721EF08F00F9A0F9C0F9E2A
:101030000101000E5E6F600E5F6F3D0E606F080E67
:10104000616F47C100F148C101F149C102F14AC1D4
:1010500003F10101140E046F050E056F000E066FFB
:10106000000E076FEEEC1EF003AF3AEF08F0F288C7
:101070005FEF08F0F2985E6B5F6B606B616B966B75
:10108000976B986B996B9A6B9B6B9C6B9D6B9E6B34
:101090009F6BA06BA16BA26BA36BA46BA56BA66BE4
:1010A000A76BA86BA96BAA6BAB6BAC6BAD6BAE6B94
:1010B000AF6BB06BB16BB26BB36BB46BB56B0CC198
:1010C00000F10DC101F10EC102F10FC103F110C118
:1010D00004F111C105F112C106F113C107F114C1E8
:1010E00008F115C109F116C10AF117C10BF135C19B
:1010F00034F10AEC23F01D661ED01CAE11D01C9EEC
:101100001D8E18AE07D0146A040E156E166A57ECC1
:1011100020F011D0146A156A166A57EC20F00BD033
:101120001CAC09D01C9C1D8C010E146E156A166A2D
:101130004BEC22F000D08BB4A5EF08F010ACA5EF7B
:1011400008F08B84109CA6EF08F08B94C3CF55F168
:10115000C4CF56F1C28207B410EF09F047C14BF17A
:1011600048C14CF149C14DF14AC14EF15EC162F135
:101170005FC163F160C164F161C165F196C1B6F10F
:1011800097C1B7F198C1B8F199C1B9F19AC1BAF153
:101190009BC1BBF19CC1BCF19DC1BDF19EC1BEF123
:1011A0009FC1BFF1A0C1C0F1A1C1C1F1A2C1C2F1F3
:1011B000A3C1C3F1A4C1C4F1A5C1C5F1A6C1C6F1C3
:1011C000A7C1C7F1A8C1C8F1A9C1C9F1AAC1CAF193
:1011D000ABC1CBF1ACC1CCF1ADC1CDF1AEC1CEF163
:1011E000AFC1CFF1B0C1D0F1B1C1D1F1B2C1D2F133
:1011F000B3C1D3F1B4C1D4F1B5C1D5F10101555199
:101200005B2756515C23E86A5D230E2E10EF09F030
:101210005CC157F15DC158F15B6B5C6B5D6B078E18
:1012200012EF09F002C0E0FF005001C0D8FF10002B
:10123000A6B218EF09F00CC0A9FF0BC0A8FFA69E2C
:10124000A69CA684F29E550EA76EAA0EA76EA68235
:10125000F28EA694A6B22AEF09F00C2A1200A96E0B
:10126000A69EA69CA680A8500C2A120004012C0E53
:10127000826F3AEC0BF0E9EC1FF00C502FEC09F008
:10128000E8CF00F10C502FEC09F0E8CF01F101AFED
:101290004FEF09F00101FF0E026FFF0E036F8CECA0
:1012A0001FF029675BEF09F00401200E826F3AEC12
:1012B0000BF060EF09F004012D0E826F3AEC0BF099
:1012C000B6EC1DF01200076A0F6A106A116A126A02
:1012D000136A0F010E0EC16E860EC06E030EC26E33
:1012E0000F01896A110E926E080E8A6EF10E936ECE
:1012F0008B6A980E946EF18EFC0E2FEC09F0E8CFFD
:101300000BF00BA011800BA211820BA411840BA86F
:101310001188C90E2FEC09F0E8CF17F0CA0E2FEC98
:1013200009F0E8CF18F0CB0E2FEC09F0E8CF19F058
:10133000CC0E2FEC09F0E8CF1AF0CD0E2FEC09F00F
:10134000E8CF2FF01C6A1D6A0E6A01015B6B5C6BB3
:101350005D6B576B586BF29A0101476B486B496B99
:101360004A6B4B6B4C6B4D6B4E6B4F6B506B516BB9
:10137000526B456B466BD76AD66A0F01280ED56E45
:10138000F28A9D90B00ECD6E01015E6B5F6B606B5B
:10139000616B626B636B646B656B666B676B686BD1
:1013A000696B536B546BCF6ACE6A0F9A0F9C0F9E7A
:1013B0009D80760ECA6E9D8202013C0E006FCC6A43
:1013C000160E2FEC09F0E8CF00F1170E2FEC09F004
:1013D000E8CF01F1180E2FEC09F0E8CF02F1190E59
:1013E0002FEC09F0E8CF03F1010103AF12EF0AF08F
:1013F000E9EC1FF0160E0C6E00C10BF018EC09F0B2
:10140000170E0C6E01C10BF018EC09F0180E0C6EE3
:1014100002C10BF018EC09F0190E0C6E03C10BF0B1
:1014200018EC09F000C18AF101C18BF102C18CF105
:1014300003C18DF100C18EF101C18FF102C190F1A4
:1014400003C191F11A0E2FEC09F0E8CF00F11B0E49
:101450002FEC09F0E8CF01F11C0E2FEC09F0E8CFDA
:1014600002F11D0E2FEC09F0E8CF03F1010103AFEB
:1014700068EF0AF0E9EC1FF01A0E0C6E00C10BF0D9
:1014800018EC09F01B0E0C6E01C10BF018EC09F002
:101490001C0E0C6E02C10BF018EC09F01D0E0C6E48
:1014A00003C10BF018EC09F01A0E2FEC09F0E8CF8D
:1014B00000F11B0E2FEC09F0E8CF01F11C0E2FEC10
:1014C00009F0E8CF02F11D0E2FEC09F0E8CF03F18F
:1014D00000C192F101C193F102C194F103C195F1F0
:1014E000240EAC6E900EAB6E240EAC6E080EB86E71
:1014F000000EB06E1F0EAF6E0401806B816B0F018A
:10150000900EAB6E0F019D8A0301806B816BC26BE5
:101510008B92146A156A166A9D8607900001F28EF6
:10152000F28C07B05FEF1CF00FB0FBEF15F010BEB0
:10153000FBEF15F012B8FBEF15F003018051811994
:101540007F0BD8B45FEF1CF013EE00F081517F0BDE
:10155000E126812BE7CFE8FFE00BD8B45FEF1CF06A
:1015600023EE82F0C2513F0BD926E7CFDFFFC22B1B
:10157000DF50780AD8A45FEF1CF007808EC100F11D
:101580008FC101F190C102F191C103F10101040E7B
:10159000046F000E056F000E066F000E076FEEEC75
:1015A0001EF000AFDDEF0AF00101030E8E6F000E9A
:1015B0008F6F000E906F000E916F03018251720ABF
:1015C000D8B4E0EF15F08251520AD8B4E0EF15F02C
:1015D0008251750AD8B4E0EF15F08251630AD8B48D
:1015E00019EF19F08251690AD8B487EF12F08251CD
:1015F0007A0AD8B49AEF13F08251490AD8B426EF88
:1016000012F08251500AD8B430EF11F08251700AB2
:10161000D8B478EF11F08251540AD8B4A8EF11F081
:101620008251740AD8B4F3EF11F08251410AD8B450
:1016300050EF0CF082514B0AD8B44EEF0BF08251B0
:101640006D0AD8B483EF10F082514D0AD8B49CEFE4
:1016500010F08251730AD8B410EF15F08251530A7A
:10166000D8B475EF15F08251590AD8B4D4EF0FF001
:1016700050EF19F0040114EE00F080517F0BE126C9
:1016800082C4E7FF802B120004010D0E826F3AEC3A
:101690000BF00A0E826F3AEC0BF0120004014B0EB5
:1016A000826F3AEC0BF004012C0E826F3AEC0BF0D7
:1016B00081B802D02FB630D003018351430AD8B489
:1016C00093EF0BF003018351630AD8B495EF0BF04D
:1016D00003018351520AD8B497EF0BF003018351F1
:1016E000720AD8B499EF0BF003018351470AD8B4BA
:1016F0009BEF0BF003018351670AD8B49DEF0BF009
:1017000003018351540AD8B49FEF0BF003018351B6
:10171000740AD8B40EEF0CF003018351550AD8B403
:10172000A1EF0BF082D02F807AD02F9078D02F822B
:1017300076D02F9274D02F8472D02F9470D02F86B1
:101740006ED084C330F185C331F186C332F187C3D3
:1017500033F10101296B37EC20F0AEEC1FF000C132
:1017600004F101C105F102C106F103C107F12AEC40
:1017700020F0200EF86EF76AF66A0900F5CF2CF11A
:101780000900F5CF2DF10900F5CF2EF10900F5CFB5
:101790002FF10900F5CF30F10900F5CF31F1090043
:1017A000F5CF32F10900F5CF33F10101296B37ECA8
:1017B00020F0AEEC1FF0EEEC1EF00067E7EF0BF050
:1017C0000167E7EF0BF00267E7EF0BF0036701D06B
:1017D00025D004014E0E826F3AEC0BF004016F0E1F
:1017E000826F3AEC0BF004014D0E826F3AEC0BF075
:1017F0000401610E826F3AEC0BF00401740E826FEB
:101800003AEC0BF00401630E826F3AEC0BF004012A
:10181000680E826F3AEC0BF04EEF19F02F96CD0E5A
:101820000C6E2FC00BF018EC09F0CD0E2FEC09F068
:10183000E8CF2FF02FB006D00401630E826F3AEC90
:101840000BF005D00401430E826F3AEC0BF02FB27F
:1018500006D00401720E826F3AEC0BF005D0040141
:10186000520E826F3AEC0BF02FB406D00401670ED3
:10187000826F3AEC0BF005D00401470E826F3AEC10
:101880000BF02FB606D00401740E826F3AEC0BF009
:1018900005D00401540E826F3AEC0BF04EEF19F0B4
:1018A0000401410E826F3AEC0BF003018351310ABF
:1018B000D8B4F4EF0EF003018351320AD8B424EF08
:1018C0000EF003018351330AD8B4ADEF0DF00301DC
:1018D0008351340AD8B49DEF0CF003018351350ACB
:1018E000D8B47AEF0CF004013F0E826F3AEC0BF0A3
:1018F0004EEF19F004012C0E826F3AEC0BF003014D
:101900008451300AD8B48DEF0CF003018451310AB0
:10191000D8B495EF0CF0E6EF0DF08B900401300E8B
:10192000826F3AEC0BF09BEF0CF08B800401310ED0
:10193000826F3AEC0BF04EEF19F0CC0E2FEC09F061
:10194000E8CF0BF004012C0E826F3AEC0BF0030190
:101950008451310AD8B4C1EF0CF003018451300A2C
:10196000D8B4C3EF0CF0030184514D0AD8B4CDEFC5
:101970000CF003018451540AD8B4D4EF0CF0EBEF0F
:101980000CF08A8401D08A940BAE04D00BAC02D048
:101990000BBA21D0E00E0B1218D01F0E0B16853992
:1019A000E844E00B0B1211D0E00E0B162AEC20F0ED
:1019B00085C332F186C333F10101296B37EC20F086
:1019C000AEEC1FF000511F0B0B12CC0E0C6E0BC0B7
:1019D0000BF018EC09F00401340E826F3AEC0BF0B6
:1019E00004012C0E826F3AEC0BF0CC0E2FEC09F0B8
:1019F000E8CF1AF08AB406D00401300E826F3AECB8
:101A00000BF005D00401310E826F3AEC0BF00401AB
:101A10002C0E826F3AEC0BF01A38E840070BE8CF37
:101A200082F40401300E82273AEC0BF004012C0EF4
:101A3000826F3AEC0BF0E9EC1FF01A501F0BE8CF65
:101A400000F18CEC1FF032C182F40401300E8227C9
:101A50003AEC0BF033C182F40401300E82273AECE9
:101A60000BF004012C0E826F3AEC0BF0E9EC1FF046
:101A70002DC000F100AF0BD0FF0E016FFF0E026F03
:101A8000FF0E036F04012D0E826F3AEC0BF08CEC0D
:101A90001FF031C182F40401300E82273AEC0BF0C2
:101AA00032C182F40401300E82273AEC0BF033C1CC
:101AB00082F40401300E82273AEC0BF004012C0E64
:101AC000826F3AEC0BF0E9EC1FF02CC000F18CECCB
:101AD0001FF031C182F40401300E82273AEC0BF082
:101AE00032C182F40401300E82273AEC0BF033C18C
:101AF00082F40401300E82273AEC0BF004012C0E24
:101B0000826F3AEC0BF0E9EC1FF02EC000F100AF51
:101B10000BD0FF0E016FFF0E026FFF0E036F04016B
:101B20002D0E826F3AEC0BF08CEC1FF031C182F479
:101B30000401300E82273AEC0BF032C182F404012A
:101B4000300E82273AEC0BF033C182F40401300EE0
:101B500082273AEC0BF04EEF19F0CB0E2FEC09F088
:101B6000E8CF0BF004012C0E826F3AEC0BF003016E
:101B70008451450AD8B4D1EF0DF003018451440AD1
:101B8000D8B4D4EF0DF003018451300AD8B4D7EFA4
:101B90000DF003018451310AD8B4DBEF0DF0E6EF0C
:101BA0000DF00B9EE0EF0DF00B8EE0EF0DF0FC0E54
:101BB0000B16E0EF0DF0FC0E0B160B80E0EF0DF0B6
:101BC000CB0E0C6E0BC00BF018EC09F00401330EB9
:101BD000826F3AEC0BF004012C0E826F3AEC0BF0A2
:101BE000CB0E2FEC09F0E8CF19F019BEFFEF0DF086
:101BF0000401450E826F3AEC0BF004EF0EF0040185
:101C0000440E826F3AEC0BF004012C0E826F3AEC1A
:101C10000BF00401300E826F3AEC0BF004012C0E35
:101C2000826F3AEC0BF019B01DEF0EF00401300E8C
:101C3000826F3AEC0BF022EF0EF00401310E826F4E
:101C40003AEC0BF04EEF19F0CA0E2FEC09F0E8CF8A
:101C50000BF004012C0E826F3AEC0BF0030184515F
:101C6000450AD8B460EF0EF003018451440AD8B499
:101C700063EF0EF0030184514D0AD8B46CEF0EF0FF
:101C800003018451410AD8B466EF0EF00301845178
:101C9000460AD8B469EF0EF003018451560AD8B44D
:101CA00074EF0EF003018451500AD8B47FEF0EF0A8
:101CB00003018451520AD8B482EF0EF08BEF0EF07C
:101CC0000B9E85EF0EF00B8E85EF0EF00B9C85EFD3
:101CD0000EF00B8C85EF0EF0FC0E0B1685C3E8FFA3
:101CE000030B0B1285EF0EF0C70E0B1685C3E8FF32
:101CF000070BE846E846E8460B1285EF0EF00B842A
:101D000085EF0EF00B9485EF0EF0CA0E0C6E0BC033
:101D10000BF018EC09F0CA0E2FEC09F0E8CF18F020
:101D20000401320E826F3AEC0BF004012C0E826F2C
:101D30003AEC0BF018BEA4EF0EF00401450E826FD2
:101D40003AEC0BF0A9EF0EF00401440E826F3AEC6E
:101D50000BF004012C0E826F3AEC0BF018C0E8FF78
:101D6000030BE8CF82F40401300E82273AEC0BF02B
:101D700004012C0E826F3AEC0BF018BCC7EF0EF08A
:101D80000401410E826F3AEC0BF0CCEF0EF004012F
:101D9000460E826F3AEC0BF004012C0E826F3AEC87
:101DA0000BF018C0E8FF380BE842E842E842E8CF01
:101DB00082F40401300E82273AEC0BF004012C0E61
:101DC000826F3AEC0BF018B4EDEF0EF00401520EF6
:101DD000826F3AEC0BF0F2EF0EF00401500E826FBE
:101DE0003AEC0BF04EEF19F0C90E2FEC09F0E8CFEA
:101DF0000BF004012C0E826F3AEC0BF003018451BE
:101E0000450AD8B412EF0FF003018451440AD8B444
:101E100015EF0FF0030184514D0AD8B418EF0FF0FD
:101E200026EF0FF00B9E20EF0FF00B8E20EF0FF040
:101E3000F80E0B1685C3E8FF070B0B1220EF0FF00F
:101E4000C90E0C6E0BC00BF018EC09F00401310E3A
:101E5000826F3AEC0BF004012C0E826F3AEC0BF01F
:101E6000C90E2FEC09F0E8CF17F017BE06D0040119
:101E7000450E826F3AEC0BF005D00401440E826FE0
:101E80003AEC0BF004012C0E826F3AEC0BF017C009
:101E9000E8FF070BE8CF82F40401300E82273AEC0A
:101EA0000BF004012C0E826F3AEC0BF00780E9EC8A
:101EB0001FF028C0E8FF003B00430043030B8CECFD
:101EC0001FF033C182F40401300E82273AEC0BF08C
:101ED00004012C0E826F3AEC0BF0E9EC1FF028C0E5
:101EE00001F1019F019D29C000F101018CEC1FF05F
:101EF0002FC182F40401300E82273AEC0BF030C17E
:101F000082F40401300E82273AEC0BF031C182F4E6
:101F10000401300E82273AEC0BF032C182F4040146
:101F2000300E82273AEC0BF033C182F40401300EFC
:101F300082273AEC0BF004012C0E826F3AEC0BF086
:101F4000E9EC1FF02AC001F12BC000F1D890013359
:101F50000033D8900133003301018CEC1FF02FC106
:101F600082F40401300E82273AEC0BF030C182F487
:101F70000401300E82273AEC0BF031C182F40401E7
:101F8000300E82273AEC0BF032C182F40401300E9D
:101F900082273AEC0BF033C182F40401300E822721
:101FA0003AEC0BF04EEF19F0FC0E2FEC09F0E8CFF5
:101FB0000BF003018351520AD8B40BEF10F0030168
:101FC0008351720AD8B40EEF10F003018351500A06
:101FD000D8B411EF10F003018351700AD8B414EF94
:101FE00010F003018351550AD8B417EF10F0030124
:101FF0008351750AD8B41AEF10F003018351430AD4
:10200000D8B423EF10F003018351630AD8B426EF4C
:1020100010F02FEF10F00B9029EF10F00B8029EF4C
:1020200010F00B9229EF10F00B8229EF10F00B94B7
:1020300029EF10F00B8429EF10F00B9629EF10F028
:102040000B8629EF10F00B9829EF10F00B8829EF81
:1020500010F0FC0E0C6E0BC00BF018EC09F0040134
:10206000590E826F3AEC0BF0119011921194119865
:10207000FC0E2FEC09F0E8CF0BF00BA011800BA2A7
:1020800011820BA411840BA8118811A04FEF10F03E
:102090000401520E826F3AEC0BF054EF10F0040181
:1020A000720E826F3AEC0BF011A85EEF10F0040193
:1020B000430E826F3AEC0BF063EF10F00401630EF5
:1020C000826F3AEC0BF011A26DEF10F00401500E8C
:1020D000826F3AEC0BF072EF10F00401700E826F19
:1020E0003AEC0BF011A47CEF10F00401550E826F56
:1020F0003AEC0BF081EF10F00401750E826F3AECB0
:102100000BF04EEF19F004016D0E826F3AEC0BF0FC
:1021100003018351300AD8B4E0EF10F0030183517A
:10212000310AD8B4F3EF10F003018351320AD8B466
:1021300006EF11F050EF19F081B803D02FB44EEF35
:1021400019F004014D0E826F3AEC0BF02AEC20F0EE
:1021500084C331F185C332F186C333F10101296BA8
:1021600037EC20F0AEEC1FF003018351300AD8B4F5
:10217000C8EF10F003018351310AD8B4D0EF10F04A
:1021800003018351320AD8B4D8EF10F050EF19F0A0
:10219000FD0E0C6E00C10BF018EC09F0E0EF10F032
:1021A000FE0E0C6E00C10BF018EC09F0F3EF10F00E
:1021B000FF0E0C6E00C10BF018EC09F006EF11F0E9
:1021C0000401300E826F3AEC0BF004012C0E826F8A
:1021D0003AEC0BF0E9EC1FF0FD0E2FEC09F0E8CF24
:1021E00000F117EF11F00401310E826F3AEC0BF0A1
:1021F00004012C0E826F3AEC0BF0E9EC1FF0FE0E9E
:102200002FEC09F0E8CF00F117EF11F00401320EC6
:10221000826F3AEC0BF0E9EC1FF004012C0E826F98
:102220003AEC0BF0FF0E2FEC09F0E8CF00F18CEC4C
:102230001FF031C182F40401300E82273AEC0BF01A
:1022400032C182F40401300E82273AEC0BF033C124
:1022500082F40401300E82273AEC0BF04EEF19F0B5
:1022600081B803D02FB226EF12F083C32AF184C3C2
:102270002BF185C32CF186C32DF187C32EF188C3C2
:102280002FF189C330F18AC331F18BC332F18CC392
:1022900033F1010137EC20F0AEEC1FF0160E0C6E9E
:1022A00000C10BF018EC09F0170E0C6E01C10BF019
:1022B00018EC09F0180E0C6E02C10BF018EC09F0C6
:1022C000190E0C6E03C10BF018EC09F000C18AF175
:1022D00001C18BF102C18CF103C18DF100C18EF1FE
:1022E00001C18FF102C190F103C191F126EF12F00B
:1022F00081B803D02FB226EF12F083C32AF184C332
:102300002BF185C32CF186C32DF187C32EF188C331
:102310002FF189C330F18AC331F18BC332F18CC301
:1023200033F1010137EC20F0AEEC1FF000C18AF16F
:1023300001C18BF102C18CF103C18DF100C18EF19D
:1023400001C18FF102C190F103C191F126EF12F0AA
:1023500081B803D02FB226EF12F083C32AF184C3D1
:102360002BF185C32CF186C32DF187C32EF188C3D1
:102370002FF189C330F18AC331F18CC332F18DC39F
:1023800033F1010137EC20F0AEEC1FF00101000E3B
:10239000046F000E056F010E066F000E076FFFEC55
:1023A0001EF01A0E0C6E00C10BF018EC09F01B0E9B
:1023B0000C6E01C10BF018EC09F01C0E0C6E02C182
:1023C0000BF018EC09F01D0E0C6E03C10BF018ECAD
:1023D00009F000C192F101C193F102C194F103C16E
:1023E00095F126EF12F081B803D02FB226EF12F04C
:1023F00083C32AF184C32BF185C32CF186C32DF14D
:1024000087C32EF188C32FF189C330F18AC331F11C
:102410008CC332F18DC333F1010137EC20F0AEEC07
:102420001FF00101000E046F000E056F010E066F14
:10243000000E076FFFEC1EF000C192F101C193F195
:1024400002C194F103C195F126EF12F0160E2FECA4
:1024500009F0E8CF00F1170E2FEC09F0E8CF01F1F9
:10246000180E2FEC09F0E8CF02F1190E2FEC09F04D
:10247000E8CF03F18CEC1FF06FEC1DF00401730E3C
:10248000826F3AEC0BF004012C0E826F3AEC0BF0E9
:102490008AC100F18BC101F18CC102F18DC103F140
:1024A0008CEC1FF06FEC1DF00401730E826F3AECA0
:1024B0000BF004012C0E826F3AEC0BF01A0E2FEC8D
:1024C00009F0E8CF00F11B0E2FEC09F0E8CF01F185
:1024D0001C0E2FEC09F0E8CF02F11D0E2FEC09F0D5
:1024E000E8CF03F16BEC19F004012C0E826F3AEC8B
:1024F0000BF092C100F193C101F194C102F195C1B9
:1025000003F16BEC19F044EC0BF050EF19F00401FF
:10251000690E826F3AEC0BF004012C0E826F3AECDC
:102520000BF00101040E006F000E016F000E026F30
:10253000000E036F8CEC1FF02CC182F40401300EEE
:1025400082273AEC0BF02DC182F40401300E822771
:102550003AEC0BF02EC182F40401300E82273AECE3
:102560000BF02FC182F40401300E82273AEC0BF0FD
:1025700030C182F40401300E82273AEC0BF031C1F5
:1025800082F40401300E82273AEC0BF032C182F45F
:102590000401300E82273AEC0BF033C182F40401BF
:1025A000300E82273AEC0BF004012C0E826F3AECCD
:1025B0000BF00101030E006F000E016F000E026FA1
:1025C000000E036F8CEC1FF02CC182F40401300E5E
:1025D00082273AEC0BF02DC182F40401300E8227E1
:1025E0003AEC0BF02EC182F40401300E82273AEC53
:1025F0000BF02FC182F40401300E82273AEC0BF06D
:1026000030C182F40401300E82273AEC0BF031C164
:1026100082F40401300E82273AEC0BF032C182F4CE
:102620000401300E82273AEC0BF033C182F404012E
:10263000300E82273AEC0BF004012C0E826F3AEC3C
:102640000BF00101300E006F000E016F000E026FE3
:10265000000E036F8CEC1FF02CC182F40401300ECD
:1026600082273AEC0BF02DC182F40401300E822750
:102670003AEC0BF02EC182F40401300E82273AECC2
:102680000BF02FC182F40401300E82273AEC0BF0DC
:1026900030C182F40401300E82273AEC0BF031C1D4
:1026A00082F40401300E82273AEC0BF032C182F43E
:1026B0000401300E82273AEC0BF033C182F404019E
:1026C000300E82273AEC0BF004012C0E826F3AECAC
:1026D0000BF0200EF86EF76AF66A04010900F5CFD8
:1026E00082F43AEC0BF00900F5CF82F43AEC0BF0EF
:1026F0000900F5CF82F43AEC0BF00900F5CF82F433
:102700003AEC0BF00900F5CF82F43AEC0BF009003B
:10271000F5CF82F43AEC0BF00900F5CF82F43AECF5
:102720000BF00900F5CF82F43AEC0BF044EC0BF01F
:1027300050EF19F081B803D02FB0EAEF13F08351B6
:10274000630AD8A44EEF19F08451610AD8A44EEF61
:1027500019F085516C0AD8A44EEF19F08651410A40
:1027600042E08651440A1BE08651420AD8B406EF83
:1027700014F08651350AD8B4DAEF1AF08651360AC9
:10278000D8B42FEF1BF08651370AD8B498EF1BF05E
:102790008651380AD8B4F6EF1BF04EEF19F00798BF
:1027A000079A04017A0E826F3AEC0BF00401780E5E
:1027B000826F3AEC0BF00401640E826F3AEC0BF07E
:1027C00081A8EAEF13F00401550E826F3AEC0BF08A
:1027D000EFEF13F004014C0E826F3AEC0BF044EC77
:1027E0000BF050EF19F00788079A04017A0E826FF8
:1027F0003AEC0BF00401410E826F3AEC0BF004014D
:10280000610E826F3AEC0BF0E0EF13F00798078A45
:1028100004017A0E826F3AEC0BF00401420E826FD3
:102820003AEC0BF00401610E826F3AEC0BF0E0EF32
:1028300013F00101666724EF14F0676724EF14F0CA
:10284000686724EF14F0696715D04F672FEF14F015
:1028500050672FEF14F051672FEF14F052670AD032
:102860000101000E006F000E016F000E026F000EDE
:10287000036F120011B80AD00101620E046F010E3D
:10288000056F000E066F000E076F09D00101A70E3D
:10289000046F020E056F000E066F000E076F66C113
:1028A00000F167C101F168C102F169C103F1EEEC09
:1028B0001EF003BFCCEF14F0119A119C0101000E21
:1028C000046FA80E056F550E066F020E076F66C1E6
:1028D00000F167C101F168C102F169C103F166C18C
:1028E00086F167C187F168C188F169C189F1EEECB1
:1028F0001EF003BF0BD00101000E866FA80E876F7C
:10290000550E886F020E896F118A119C0E0E2FECE6
:1029100009F0E8CF18F10F0E2FEC09F0E8CF19F10C
:10292000100E2FEC09F0E8CF1AF1110E2FEC09F080
:10293000E8CF1BF137EC1EF086C104F187C105F129
:1029400088C106F189C107F1EEEC1EF00782FBECAD
:102950001DF037EC1EF00792FBEC1DF086C100F174
:1029600087C101F188C102F189C103F10792FBEC33
:102970001DF0CC0E046FE00E056F870E066F050E7E
:10298000076FEEEC1EF000C118F101C119F102C190
:102990001AF103C11BF13BD0119C119A0101800E69
:1029A000006F1A0E016F060E026F000E036F4FC10B
:1029B00004F150C105F151C106F152C107F1EEEC2D
:1029C0001EF003AF05D0E9EC1FF0118C119A120034
:1029D0000E0E2FEC09F0E8CF18F10F0E2FEC09F0D6
:1029E000E8CF19F1100E2FEC09F0E8CF1AF1110E13
:1029F0002FEC09F0E8CF1BF14FC100F150C101F1FC
:102A000051C102F152C103F10782FBEC1DF018C164
:102A100000F119C101F11AC102F11BC103F1120049
:102A20000401730E826F3AEC0BF004012C0E826FDE
:102A30003AEC0BF0078462C166F163C167F164C1CF
:102A400068F165C169F14BC14FF14CC150F14DC105
:102A500051F14EC152F157C159F158C15AF1079481
:102A600036EC15F044EC0BF050EF19F066C100F1B4
:102A700067C101F168C102F169C103F101018CEC88
:102A80001FF06FEC1DF00401630E826F3AEC0BF047
:102A900004012C0E826F3AEC0BF04FC100F150C1D3
:102AA00001F151C102F152C103F101018CEC1FF09F
:102AB0006FEC1DF00401660E826F3AEC0BF004011E
:102AC0002C0E826F3AEC0BF0E9EC1FF059C100F1CB
:102AD0005AC101F101018CEC1FF06FEC1DF00401F3
:102AE000740E826F3AEC0BF0120010820401530E48
:102AF000826F3AEC0BF004012C0E826F3AEC0BF073
:102B000083C32AF184C32BF185C32CF186C32DF135
:102B100087C32EF188C32FF189C330F18AC331F105
:102B20008BC332F18CC333F1010137EC20F0AEECF2
:102B30001FF000C166F101C167F102C168F103C174
:102B400069F18EC32AF18FC32BF190C32CF191C38D
:102B50002DF192C32EF193C32FF194C330F195C39D
:102B600031F196C332F197C333F1010137EC20F014
:102B7000AEEC1FF000C14FF101C150F102C151F1A3
:102B800003C152F12AEC20F099C32FF19AC330F11E
:102B90009BC331F19CC332F19DC333F1010137EC8A
:102BA00020F0AEEC1FF000C159F101C15AF136EC32
:102BB00015F004012C0E826F3AEC0BF0EFEF15F0DC
:102BC000118E19A002D019AE108C18BE02D018A414
:102BD000108E8251520A02E10F8201D00F9282516F
:102BE000750A02E1108401D010948251550A02E165
:102BF000108601D0109611A003D011A401D010842A
:102C0000078410B25DEF16F010A449EF16F0B6C1BC
:102C100066F1B7C167F1B8C168F1B9C169F1BAC16C
:102C20006AF1BBC16BF1BCC16CF1BDC16DF1BEC13C
:102C30006EF1BFC16FF1C0C170F1C1C171F1C2C10C
:102C400072F1C3C173F1C4C174F1C5C175F1C6C1DC
:102C500076F1C7C177F1C8C178F1C9C179F1CAC1AC
:102C60007AF1CBC17BF1CCC17CF1CDC17DF1CEC17C
:102C70007EF1CFC17FF1D0C180F1D1C181F1D2C14C
:102C800082F1D3C183F1D4C184F1D5C185F151EF73
:102C900016F062C166F163C167F164C168F165C194
:102CA00069F14BC14FF14CC150F14DC151F14EC1D1
:102CB00052F157C159F158C15AF107940FA07FEF53
:102CC00016F0010192676CEF16F093676CEF16F047
:102CD00094676CEF16F0956770EF16F07FEF16F0C3
:102CE00019EC14F092C104F193C105F194C106F1FD
:102CF00095C107F1EEEC1EF003BF16EF19F019ECC9
:102D000014F00101000E046F000E056F010E066F36
:102D1000000E076F1FEC1FF011A02CD011A22AD0BB
:102D20008CEC1FF0296701D007D004012D0E826FB3
:102D30003AEC0BF014EF19F030C182F40401300EBC
:102D400082273AEC0BF031C182F40401300E822765
:102D50003AEC0BF032C182F40401300E82273AECD7
:102D60000BF033C182F40401300E82273AEC0BF0F1
:102D700014EF19F012A8C5D012981AC01BF01B3A14
:102D80001B42070E1B1600011B50000AD8B44DEF62
:102D900017F000011B50010AD8B4D9EF16F000015A
:102DA0001B50020AD8B4D7EF16F07FEF17F07FEF71
:102DB00017F0E9EC1FF02AC001F12BC000F1D89008
:102DC00001330033D890013300330101630E046FE7
:102DD000000E056F000E066F000E076F1FEC1FF050
:102DE000280E046F000E056F000E066F000E076FB1
:102DF000EEEC1EF000C12DF0E9EC1FF028C001F14F
:102E0000019F019D29C000F10101A40E046F000E75
:102E1000056F000E066F000E076F1FEC1FF000C15C
:102E20002CF000C104F101C105F102C106F103C19A
:102E300007F1640E006F000E016F000E026F000EAE
:102E4000036FEEEC1EF0050E046F000E056F000E12
:102E5000066F000E076F1FEC1FF000C104F101C1E7
:102E600005F102C106F103C107F1E9EC1FF02DC025
:102E700000F1EEEC1EF000C12EF02EC0E8FF050FB1
:102E80002D5C03E78A847FEF17F02EC0E8FF0A0F5E
:102E90002D5C01E68A947FEF17F000C124F101C197
:102EA00025F102C126F103C127F1E9EC1FF0EFEC97
:102EB0001FF01A501F0BE8CF00F10101640E046FE0
:102EC000000E056F000E066F000E076FFFEC1EF080
:102ED00024C104F125C105F126C106F127C107F17E
:102EE000EEEC1EF003BF02D08A9401D08A8424C184
:102EF00000F125C101F126C102F127C103F116EF4E
:102F000019F000C124F101C125F102C126F103C16C
:102F100027F110AE4CD0109E00C108F101C109F19B
:102F200002C10AF103C10BF18CEC1FF030C1D6F1E4
:102F300031C1D7F132C1D8F133C1D9F108C100F1A3
:102F400009C101F10AC102F10BC103F101016C0ECB
:102F5000046F070E056F000E066F000E076FEEEC94
:102F60001EF003BF04D00101550EDA6F1CD008C15A
:102F700000F109C101F10AC102F10BC103F1010124
:102F8000A40E046F060E056F000E066F000E076F8D
:102F9000EEEC1EF003BF04D001017F0EDA6F03D008
:102FA0000101FF0EDA6F1C8E11AE16EF19F024C16D
:102FB00000F125C101F126C102F127C103F110A4DE
:102FC000E9EF17F00401750E826F3AEC0BF0EEEFAB
:102FD00017F00401720E826F3AEC0BF004012C0E14
:102FE000826F3AEC0BF08CEC1FF02967FDEF17F0C5
:102FF0000401200E826F00EF18F004012D0E826F85
:103000003AEC0BF030C182F40401300E82273AEC26
:103010000BF031C182F40401300E82273AEC0BF040
:1030200004012E0E826F3AEC0BF032C182F40401DF
:10303000300E82273AEC0BF033C182F40401300EDB
:1030400082273AEC0BF004016D0E826F3AEC0BF024
:1030500004012C0E826F3AEC0BF04FC100F150C10D
:1030600001F151C102F152C103F101018CEC1FF0D9
:103070006FEC1DF00401480E826F3AEC0BF0040176
:103080007A0E826F3AEC0BF004012C0E826F3AEC50
:103090000BF066C100F167C101F168C102F169C1BD
:1030A00003F101018CEC1FF06FEC1DF00401630EC5
:1030B000826F3AEC0BF004012C0E826F3AEC0BF0AD
:1030C00066C100F167C101F168C102F169C103F194
:1030D00001010A0E046F000E056F000E066F000E50
:1030E000076FFFEC1EF0000E046F120E056F000E4E
:1030F000066F000E076F1FEC1FF08CEC1FF02AC14B
:1031000082F40401300E82273AEC0BF02BC182F4DA
:103110000401300E82273AEC0BF02CC182F404013A
:10312000300E82273AEC0BF02DC182F40401300EF0
:1031300082273AEC0BF02EC182F40401300E822774
:103140003AEC0BF02FC182F40401300E82273AECE6
:103150000BF030C182F40401300E82273AEC0BF000
:1031600004012E0E826F3AEC0BF031C182F404019F
:10317000300E82273AEC0BF032C182F40401300E9B
:1031800082273AEC0BF033C182F40401300E82271F
:103190003AEC0BF00401730E826F3AEC0BF0040171
:1031A0002C0E826F3AEC0BF0E9EC1FF059C100F1E4
:1031B0005AC101F17AEC1AF00FB2E2EF18F00FA049
:1031C00014EF19F004012C0E826F3AEC0BF0200E74
:1031D000F86EF76AF66A04010900F5CF82F43AEC5A
:1031E0000BF00900F5CF82F43AEC0BF00900F5CFB3
:1031F00082F43AEC0BF00900F5CF82F43AEC0BF0D4
:103200000900F5CF82F43AEC0BF00900F5CF82F417
:103210003AEC0BF00900F5CF82F43AEC0BF0090020
:10322000F5CF82F43AEC0BF044EC0BF00F9050EF3A
:1032300019F00401630E826F3AEC0BF004012C0EBE
:10324000826F3AEC0BF056EC19F004012C0E826FF1
:103250003AEC0BF0C9EC19F004012C0E826F3AEC39
:103260000BF045EC1AF004012C0E826F3AEC0BF0D7
:103270000101F80E006FCD0E016F660E026F030E96
:10328000036F6BEC19F004012C0E826F3AEC0BF01B
:103290005BEC1AF044EC0BF050EF19F044EC0BF03F
:1032A0000301C26B079010925FEF1CF0D8900E0ED6
:1032B0002FEC09F0E8CF00F10F0E2FEC09F0E8CF6A
:1032C00001F1100E2FEC09F0E8CF02F1110E2FECF6
:1032D00009F0E8CF03F10101000E046F000E056F45
:1032E000010E066F000E076F1FEC1FF08CEC1FF035
:1032F0002AC182F40401300E82273AEC0BF02BC174
:1033000082F40401300E82273AEC0BF02CC182F4D7
:103310000401300E82273AEC0BF02DC182F4040137
:10332000300E82273AEC0BF02EC182F40401300EED
:1033300082273AEC0BF02FC182F40401300E822771
:103340003AEC0BF030C182F40401300E82273AECE3
:103350000BF031C182F40401300E82273AEC0BF0FD
:1033600004012E0E826F3AEC0BF032C182F404019C
:10337000300E82273AEC0BF033C182F40401300E98
:1033800082273AEC0BF004016D0E826F3AEC0BF0E1
:103390001200120E2FEC09F0E8CF00F1130E2FEC03
:1033A00009F0E8CF01F1140E2FEC09F0E8CF02F19B
:1033B000150E2FEC09F0E8CF03F101010A0E046F9E
:1033C000000E056F000E066F000E076FFFEC1EF07B
:1033D000000E046F120E056F000E066F000E076FD1
:1033E0001FEC1FF08CEC1FF02AC182F40401300E98
:1033F00082273AEC0BF02BC182F40401300E8227B5
:103400003AEC0BF02CC182F40401300E82273AEC26
:103410000BF02DC182F40401300E82273AEC0BF040
:103420002EC182F40401300E82273AEC0BF02FC13A
:1034300082F40401300E82273AEC0BF030C182F4A2
:103440000401300E82273AEC0BF004012E0E826F3D
:103450003AEC0BF031C182F40401300E82273AECD1
:103460000BF032C182F40401300E82273AEC0BF0EB
:1034700033C182F40401300E82273AEC0BF00401D0
:10348000730E826F3AEC0BF012000A0E2FEC09F06B
:10349000E8CF00F10B0E2FEC09F0E8CF01F10C0E94
:1034A0002FEC09F0E8CF02F10D0E2FEC09F0E8CF78
:1034B00003F17AEF1AF0060E2FEC09F0E8CF00F1D5
:1034C000070E2FEC09F0E8CF01F1080E2FEC09F000
:1034D000E8CF02F1090E2FEC09F0E8CF03F17AEF03
:1034E0001AF00101E9EC1FF0078457C100F158C13F
:1034F00001F107940101E80E046F800E056F000EC4
:10350000066F000E076FFFEC1EF0000E046F040E36
:10351000056F000E066F000E076F1FEC1FF0880E80
:10352000046F130E056F000E066F000E076FEEECB2
:103530001EF00A0E046F000E056F000E066F000EDF
:10354000076F1FEC1FF08CEC1FF001012967AEEF35
:103550001AF00401200E826FB1EF1AF004012D0E53
:10356000826F3AEC0BF030C182F40401300E8227F6
:103570003AEC0BF031C182F40401300E82273AECB0
:103580000BF032C182F40401300E82273AEC0BF0CA
:1035900004012E0E826F3AEC0BF033C182F4040169
:1035A000300E82273AEC0BF00401430E826F3AECA6
:1035B0000BF0120087C32AF188C32BF189C32CF1C9
:1035C0008AC32DF18BC32EF18CC32FF18DC330F143
:1035D0008EC331F190C332F191C333F10101296BF4
:1035E00037EC20F0AEEC1FF00101000E046F000E6E
:1035F000056F010E066F000E076FFFEC1EF00E0E3A
:103600000C6E00C10BF018EC09F00F0E0C6E01C12E
:103610000BF018EC09F0100E0C6E02C10BF018EC58
:1036200009F0110E0C6E03C10BF018EC09F0040147
:103630007A0E826F3AEC0BF004012C0E826F3AEC9A
:103640000BF00401350E826F3AEC0BF004012C0EE6
:10365000826F3AEC0BF056EC19F0EFEF13F087C3E2
:103660002AF188C32BF189C32CF18AC32DF18BC3B6
:103670002EF18CC32FF18DC330F18EC331F190C385
:1036800032F191C333F10101296B37EC20F0AEEC3C
:103690001FF0880E046F130E056F000E066F000EEC
:1036A000076FF3EC1EF0000E046F040E056F000EA2
:1036B000066F000E076FFFEC1EF00101E80E046FAD
:1036C000800E056F000E066F000E076F1FEC1FF0D7
:1036D0000A0E0C6E00C10BF018EC09F00B0E0C6E0C
:1036E00001C10BF018EC09F00C0E0C6E02C10BF0CE
:1036F00018EC09F00D0E0C6E03C10BF018EC09F07C
:1037000004017A0E826F3AEC0BF004012C0E826FEA
:103710003AEC0BF00401360E826F3AEC0BF0040128
:103720002C0E826F3AEC0BF045EC1AF0EFEF13F031
:1037300087C32AF188C32BF189C32CF18AC32DF1E9
:103740008BC32EF18CC32FF18DC330F18FC331F1B8
:1037500090C332F191C333F1010137EC20F0AEECAC
:103760001FF0000E046F120E056F000E066F000EA4
:10377000076FFFEC1EF001010A0E046F000E056FCB
:10378000000E066F000E076F1FEC1FF0120E0C6E7E
:1037900000C10BF018EC09F0130E0C6E01C10BF018
:1037A00018EC09F0140E0C6E02C10BF018EC09F0C5
:1037B000150E0C6E03C10BF018EC09F004017A0E23
:1037C000826F3AEC0BF004012C0E826F3AEC0BF096
:1037D0000401370E826F3AEC0BF004012C0E826F5D
:1037E0003AEC0BF0C9EC19F0EFEF13F087C32AF1B4
:1037F00088C32BF189C32CF18AC32DF18BC32EF121
:103800008CC32FF18DC330F18EC331F190C332F1EF
:1038100091C333F10101296B37EC20F0AEEC1FF0BE
:10382000880E046F130E056F000E066F000E076FF3
:10383000F3EC1EF0000E046F040E056F000E066F11
:10384000000E076FFFEC1EF00101E80E046F800E02
:10385000056F000E066F000E076F1FEC1FF0060EBF
:103860000C6E00C10BF018EC09F0070E0C6E01C1D4
:103870000BF018EC09F0080E0C6E02C10BF018ECFE
:1038800009F0090E0C6E03C10BF018EC09F00401ED
:103890007A0E826F3AEC0BF004012C0E826F3AEC38
:1038A0000BF00401380E826F3AEC0BF004012C0E81
:1038B000826F3AEC0BF05BEC1AF0EFEF13F081B88B
:1038C00003D02FB01DEF1DF007A8D7EF1CF00101AA
:1038D000800E006F1A0E016F060E026F000E036F4E
:1038E0004BC104F14CC105F14DC106F14EC107F1C8
:1038F000EEEC1EF003BF1DEF1DF069EC1DF04BC197
:1039000000F14CC101F14DC102F14EC103F107823A
:10391000FBEC1DF018C104F119C105F11AC106F143
:103920001BC107F1F80E006FCD0E016F660E026F1E
:10393000030E036FEEEC1EF00E0E0C6E00C10BF0CA
:1039400018EC09F00F0E0C6E01C10BF018EC09F029
:10395000100E0C6E02C10BF018EC09F0110E0C6E7B
:1039600003C10BF018EC09F007840101E9EC1FF02A
:1039700057C100F158C101F107940A0E0C6E00C145
:103980000BF018EC09F00B0E0C6E01C10BF018ECEB
:1039900009F00C0E0C6E02C10BF018EC09F00D0EC4
:1039A0000C6E03C10BF018EC09F01DEF1DF007AA17
:1039B0001DEF1DF007840101E9EC1FF057C100F174
:1039C00058C101F10794060E0C6E00C10BF018EC03
:1039D00009F0070E0C6E01C10BF018EC09F0080E8F
:1039E0000C6E02C10BF018EC09F0090E0C6E03C14D
:1039F0000BF018EC09F0078462C100F163C101F11A
:103A000064C102F165C103F10794120E0C6E00C18E
:103A10000BF018EC09F0130E0C6E01C10BF018EC52
:103A200009F0140E0C6E02C10BF018EC09F0150E23
:103A30000C6E03C10BF018EC09F00798079A04010B
:103A4000805181197F0B0DE09EA8FED714EE00F087
:103A500081517F0BE126E750812B0F01AD6E1FEFE7
:103A60001DF091EF0AF018C100F119C101F11AC15E
:103A700002F11BC103F1000E046F000E056F010E71
:103A8000066F000E076F1FEC1FF029A15EEF1DF0FF
:103A90002051D8B45EEF1DF018C100F119C101F139
:103AA0001AC102F11BC103F1000E046F000E056F75
:103AB0000A0E066F000E076F1FEC1FF012000101C7
:103AC000045100130551011306510213075103134A
:103AD00012000101186B196B1A6B1B6B12002AC1C3
:103AE00082F40401300E82273AEC0BF02BC182F4F1
:103AF0000401300E82273AEC0BF02CC182F4040151
:103B0000300E82273AEC0BF02DC182F40401300E06
:103B100082273AEC0BF02EC182F40401300E82278A
:103B20003AEC0BF02FC182F40401300E82273AECFC
:103B30000BF030C182F40401300E82273AEC0BF016
:103B400031C182F40401300E82273AEC0BF032C10D
:103B500082F40401300E82273AEC0BF033C182F478
:103B60000401300E82273AEC0BF012002FC182F4D0
:103B70000401300E82273AEC0BF030C182F40401CC
:103B8000300E82273AEC0BF031C182F40401300E82
:103B900082273AEC0BF032C182F40401300E822706
:103BA0003AEC0BF033C182F40401300E82273AEC78
:103BB0000BF01200060E1E6E060E1F6E060E206E15
:103BC0001E2EE0EF1DF01F2EE0EF1DF0202EE0EF87
:103BD0001DF08B84020E1E6E020E1F6E020E206EF2
:103BE0001E2EF0EF1DF01F2EF0EF1DF0202EF0EF37
:103BF0001DF08B9412000101005305E1015303E114
:103C0000025301E1002BBEEC1EF0E9EC1FF039512C
:103C1000006F3A51016F420E046F4B0E056F000E9C
:103C2000066F000E076FFFEC1EF000C104F101C12A
:103C300005F102C106F103C107F118C100F119C174
:103C400001F11AC102F11BC103F107B22CEF1EF002
:103C5000F3EC1EF02EEF1EF0EEEC1EF000C118F19A
:103C600001C119F102C11AF103C11BF11200E9EC03
:103C70001FF059C100F15AC101F1060E2FEC09F0F5
:103C8000E8CF04F1070E2FEC09F0E8CF05F1080E9C
:103C90002FEC09F0E8CF06F1090E2FEC09F0E8CF80
:103CA00007F1EEEC1EF000C124F101C125F102C1C3
:103CB00026F103C127F1290E046F000E056F000ED7
:103CC000066F000E076FFFEC1EF0EE0E046F430E42
:103CD000056F000E066F000E076FF3EC1EF024C197
:103CE00004F125C105F126C106F127C107F1FFEC5A
:103CF0001EF000C11CF101C11DF102C11EF103C182
:103D00001FF1120E2FEC09F0E8CF04F1130E2FEC87
:103D100009F0E8CF05F1140E2FEC09F0E8CF06F119
:103D2000150E2FEC09F0E8CF07F10D0E006F000E15
:103D3000016F000E026F000E036FFFEC1EF0180EF5
:103D4000046F000E056F000E066F000E076F1FEC6C
:103D50001FF01CC104F11DC105F11EC106F11FC1F8
:103D600007F1F3EC1EF06A0E046F2A0E056F000EC9
:103D7000066F000E076FEEEC1EF01200BF0EFA6E1B
:103D8000200E3A6F396BD89000370137023703376E
:103D9000D8B0CFEF1EF03A2FC4EF1EF039073A0724
:103DA0000353D8B412000331070B80093F6F033966
:103DB0000F0B010F396F80EC5FF0406F390580EC1D
:103DC0005FF0405D405F396B3F33D8B039273933FE
:103DD0003FA9E4EF1EF040513927120001010EEC1B
:103DE00020F0D8B01200010103510719346FD1EC53
:103DF0001FF0D8900751031934AF800F1200010152
:103E0000346BF5EC1FF0D8A00BEC20F0D8B012000A
:103E1000E0EC1FF0E9EC1FF01F0E366F21EC20F0F4
:103E20000B35D8B0D1EC1FF0D8A00335D8B01200B4
:103E3000362F0EEF1FF034B1F8EC1FF01200010125
:103E4000346B04510511061107110008D8A0F5ECD8
:103E50001FF0D8A00BEC20F0D8B01200086B096B53
:103E60000A6B0B6B21EC20F01F0E366F21EC20F05B
:103E700007510B5DD8A449EF1FF006510A5DD8A485
:103E800049EF1FF00551095DD8A449EF1FF0045117
:103E9000085DD8A05CEF1FF00451085F0551D8A061
:103EA000053D095F0651D8A0063D0A5F0751D8A01D
:103EB000073D0B5FD8900081362F36EF1FF034B1ED
:103EC000F8EC1FF0346BF5EC1FF0D89025EC20F0E7
:103ED00007510B5DD8A479EF1FF006510A5DD8A4F5
:103EE00079EF1FF00551095DD8A479EF1FF0045157
:103EF000085DD8A088EF1FF0003F88EF1FF0013F5A
:103F000088EF1FF0023F88EF1FF0032BD8B4120098
:103F100034B1F8EC1FF012000101346BF5EC1FF026
:103F2000D8B012002AEC20F0200E366F003701378F
:103F30000237033711EE33F00A0E376FE7360A0EF9
:103F4000E75CD8B0E76EE552372F9EEF1FF0362FB3
:103F500096EF1FF034B12981D890120001010A0EAA
:103F6000346F200E366F11EE29F03451376F0A0E80
:103F7000D890E652D8B0E726E732372FB9EF1FF0D6
:103F80000333023301330033362FB3EF1FF0E75012
:103F9000FF0FD8A00335D8B0120029B1F8EC1FF0FC
:103FA0001200045100270551D8B0053D01270651E4
:103FB000D8B0063D02270751D8B0073D03271200AD
:103FC0000051086F0151096F02510A6F03510B6FC5
:103FD00012000101006B016B026B036B1200010107
:103FE000046B056B066B076B12000335D8A012003B
:103FF0000351800B001F011F021F031F003F08EF2A
:1040000020F0013F08EF20F0023F08EF20F0032BE3
:10401000342B032512000735D8A012000751800B5E
:10402000041F051F061F071F043F1EEF20F0053F5A
:104030001EEF20F0063F1EEF20F0072B342B072544
:1040400012000037013702370337083709370A37BC
:104050000B3712000101296B2A6B2B6B2C6B2D6B1C
:104060002E6B2F6B306B316B326B336B1200010197
:104070002A510F0B2A6F2B510F0B2B6F2C510F0B4B
:104080002C6F2D510F0B2D6F2E510F0B2E6F2F51AB
:104090000F0B2F6F30510F0B306F31510F0B316FF2
:1040A00032510F0B326F33510F0B336F120000017F
:1040B0001650FF0A01E11200390EC86E800EC76E5D
:1040C000280EC66E000EC56E1550000AD8B492EFC9
:1040D00020F01550010AD8B4ABEF20F01550020AB9
:1040E000D8B4C4EF20F01550030AD8B4DDEF20F0A7
:1040F0001550040AD8B405EF21F01550050AD8B4BC
:104100001EEF21F01550060AD8B437EF21F01550F4
:10411000070AD8B450EF21F01550080AD8B469EF57
:1041200021F012001650000AD8B488EF21F0165082
:10413000010AD8B48CEF21F01650020AD8B490EFDF
:1041400021F01650030AD8B494EF21F01650040A57
:10415000D8B403EF22F01650000AD8B498EF21F03B
:104160001650010AD8B49CEF21F01650020AD8B4B8
:10417000A0EF21F01650030AD8B4A4EF21F0165096
:10418000040AD8B403EF22F01650000AD8B4A8EFFE
:1041900021F01650010AD8B4ACEF21F01650020AF3
:1041A000D8B4B0EF21F01650030AD8B4B4EF21F020
:1041B0001650040AD8B403EF22F01650000AD8B4FF
:1041C000C1EF21F01650010AD8B4C5EF21F0165006
:1041D000020AD8B4C9EF21F01650030AD8B4DDEFB3
:1041E00021F01650040AD8B4E1EF21F01650050A68
:1041F000D8B4E5EF21F01650060AD8B4E9EF21F063
:104200001650070AD8B4ECEF21F01650000AD8B4C3
:10421000F0EF21F01650010AD8B4F4EF21F0165057
:10422000020AD8B4F8EF21F01650030AD8B4FCEF14
:1042300021F01650040AD8B4FFEF21F01650000AFE
:10424000D8B407EF22F01650010AD8B40BEF22F0D1
:104250001650020AD8B40FEF22F01650030AD8B451
:1042600013EF22F01650040AD8B403EF22F01650D0
:10427000000AD8B41DEF22F01650010AD8B421EF7D
:1042800022F01650020AD8B425EF22F01650030A85
:10429000D8B429EF22F01650040AD8B403EF22F064
:1042A0001650000AD8B42AEF22F01650010AD8B4EA
:1042B0002EEF22F01650020AD8B432EF22F0165038
:1042C000030AD8B436EF22F01650040AD8B403EF2C
:1042D00022F01650000AD8B437EF22F01650010A27
:1042E000D8B43BEF22F01650020AD8B43FEF22F0C8
:1042F0001650030AD8B443EF22F01650040AD8B47B
:1043000044EF22F01650050AD8B447EF22F012000D
:104310009E96C580162A1200E20EC96E162A120059
:10432000770EC96E162A1200020EC96E162A1200E6
:104330009E96C580162A1200E20EC96E162A120039
:10434000790EC96E162A1200000EC96E162A1200C6
:104350009E96C580162A1200E20EC96E162A120019
:104360007A0EC96E162A120018BC03D0DAC1E8FF13
:1043700004D01850E844E8441F09E8CFC9FF162AC2
:1043800012009E96C580162A1200E20EC96E162AE9
:10439000120011BA03D011BC01D003D0050E156E66
:1043A0003ED00101D667D9EF21F0100EC96EDBEFC8
:1043B00021F0D6C1C9FF162A1200D7C1C9FF162A9B
:1043C0001200D8C1C9FF162A1200D9C1C9FF162A86
:1043D0001200C584162A1200FF0E166E1D9E1200D2
:1043E0009E96C580162A1200E20EC96E162A120089
:1043F000760EC96E162A1200C584162A1200FF0E08
:10440000166E1D9E1200C584152A166A12009E960D
:10441000C580162A1200E20EC96E162A12007B0E03
:10442000C96E162A120011AA04D0230EC96E162ACC
:1044300012001C0EC96E162A12009E96C580162AFE
:104440001200E20EC96E162A12007C0EC96E162AE0
:104450001200E9D79E96C580162A1200E20EC96E98
:10446000162A12007D0EC96E162A1200DCD79E96FF
:10447000C580162A1200E20EC96E162A12007E0EA0
:10448000C96E162A1200CFD7C584162A1200FF0E55
:10449000166E1D9E12001650FF0AD8B409EF23F0C5
:1044A000390EC86E800EC76E280EC66E000EC56E21
:1044B0001550000AD8B464EF22F01550010AD8B4A0
:1044C00078EF22F009EF23F01650000AD8B4B6EFC7
:1044D00022F01650010AD8B4BAEF22F01650020AA0
:1044E000D8B4C4EF22F01650030AD8B4C7EF22F0B4
:1044F0001650000AD8B4CDEF22F01650010AD8B4F5
:10450000D1EF22F01650020AD8B4DBEF22F0165099
:10451000030AD8B4DEEF22F01650040AD8B4E4EF50
:1045200022F01650050AD8B4E7EF22F01650060A1A
:10453000D8B4EDEF22F01650070AD8B4F0EF22F00D
:104540001650080AD8B4F6EF22F01650090AD8B46B
:10455000F9EF22F016500A0AD8B4FFEF22F01650F5
:104560000B0AD8B402EF23F009EF23F09E96C58022
:1045700008EF23F017B004D04E0EC96E08EF23F0F9
:10458000500EC96E08EF23F0C58408EF23F0152AFA
:10459000FF0E166E128009EF23F09E96C58008EF7D
:1045A00023F017B004D04F0EC96E08EF23F0510E60
:1045B000C96E08EF23F0C58608EF23F0C9CF24F0B9
:1045C000C59AC58808EF23F0C58608EF23F0C9CF48
:1045D00025F0C59AC58808EF23F0C58608EF23F0BB
:1045E000C9CF26F0C59AC58808EF23F0C58608EF25
:1045F00023F0C9CF27F0C58AC58808EF23F0C5840A
:1046000008EF23F0FF0E166E12861D9C09EF23F0B3
:10461000162A120012B012D012B213D012B414D053
:1046200012A6120007B01200129624C028F025C06E
:1046300029F026C02AF027C02BF012001290128217
:10464000120012921284120000011650FF0A04E1B7
:0A4650001294166A4BEC22F01200DF
:10BF0000E844F926000C160C2B0C3F0C520C640C68
:10BF1000760C860C960CA50CB30CC10CCF0CDC0C6B
:06BF2000E80CF40C000C1B
:00000001FF
